:1000000036C052C051C050C04FC057C04DC04CC088
:100010004BC04AC049C048C047C046C045C08BA27B
:10002000B0B9C2FF010A2A4B7A85FF010203050716
:10003000EEF3F400010203050700070503020100C7
:10004000020407EEF3F4F0000204070007040200C4
:1000500001020306EEF3F4F00001020306000603BA
:1000600002010002030507000704EE000700112447
:100070001FBECFE5D2E0DEBFCDBF20E0A0E6B0E0FE
:1000800001C01D92A137B207E1F7E2E7F0E012826A
:10009000108688E58187E0E6F0E08DEF87838EEFBC
:1000A0008583712C94D0C7C1ABCF8150E82FF0E08D
:1000B000EC5DFF4FE491E9BD0895189525B7277EC3
:1000C00025BF29B7226029BF21E022BF019728F070
:1000D00020E188952150E9F7F9CF089588EE93E063
:1000E000EDCF369A3699FECF85B108958091710093
:1000F000EEE7F0E08083818382830895CF93C72D5C
:1001000081E0870D8F73782E662D90E086D16FEF9A
:100110008C2F90E0CF9181C1FF920F931F93CF93CB
:10012000DF93F82E03E710E0CEE7D0E0F11005C032
:10013000CE016BD1F801808304C0F8016081CE014B
:100140006CD121970F5F1F4FC537D10579F7DF912C
:10015000CF911F910F91FF900895D0DF81E0DCCF08
:10016000811102C019BC0895A0CF0F931F93CF93A4
:10017000C82F8B01CC2359F081E097DFC8019EDFA7
:1001800019BCC8019BDFC80199DFC150F3CFCF91E3
:100190001F910F9108951F93CF93DF938FEA87B933
:1001A00086EC86B910E1C0E0D0E085E090E086DF23
:1001B00098DFC80FD11D1150C1F7CE0124E09695EC
:1001C00087952A95E1F7DF91CF911F9108951092BD
:1001D0007100712C872D90E018D1682E8F3F31F07F
:1001E0008FEF68120AC0612CB8DF09C0872D91E03B
:1001F000970D792E803470F3F3CF80E08DDF9091EE
:100200007A009F5F20E06BE270E0992399F0AB01E8
:100210004F5F5F4FFA013197E491A22FB0E0A859E8
:10022000BF4FEC93EE2319F0242F261BF1CF9150F2
:10023000BA01EBCF20937C0020937D00962D953F53
:10024000E8F48091800030917F008313D0C030911A
:100250007E008313CCC08F3F09F0D0C047DF809170
:100260007E008F5F80937E0080917F008F5F809300
:100270007F00809180008F5F809380008FE384BB3C
:1002800081E087BB9AEF98BB83BF81E88ABD85B7C1
:10029000806285BF789481EA87B986EC86B9C62DDD
:1002A000C53F10F0612C34C080917E00803138F45D
:1002B000E62DF0E0E859FF4FC081DC2F29C00EDFAA
:1002C00015DFC3E7D0E000E010E0FF24F39481E005
:1002D000800F0F5F1F4F98819F3FA9F06DE570E081
:1002E00044DFF801E05AFF4F608088818F258883C2
:1002F00034DF6FE070E080E238DF88818F2588830B
:10030000612C2BDFEBDE21960730110501F7D0CFF2
:10031000F5DE10E081EAF82E96ECE92EDD24DA9481
:10032000CE3E69F408E087E0C0DE81E290E0C6DE00
:1003300019BC83E490E0C2DE0150A9F756C0C33F68
:1003400041F487E0B2DE8AE090E0B8DE88E0ADDE1E
:1003500023C0C43F79F4C5DE90E0E92FF0E0E25E0F
:10036000FF4FE491E81710F49F5FF7CF6DE770E05F
:10037000892F10C0CE3F91F410927A00EEDE6AEF22
:1003800070E081E0F2DE81E080937A00E6DE6AEFE1
:1003900070E081E0EADEA2DEA1DE27C0CD3F89F475
:1003A0008FEF80937B00D9DE81E07FDE97DE96DEE3
:1003B00087E07BDEF0DE80937B00CFDE8FDE8EDE9B
:1003C000F9CF8D2FCDDEE7DEF7B8E6B81F5F90914D
:1003D0007B00891738F0D43028F0153118F0D0920E
:1003E0007100D3E084EF91E069DE80DE99CF7EDE9C
:1003F00080917400811142CF612C40CF9F5F692EA4
:10040000921708F42CCF612C2ACFE199FECF9FBB25
:100410008EBBE09A99278DB30895262FE199FECFE0
:100420001CBA9FBB8EBB2DBB0FB6F894E29AE19A23
:0A0430000FBE01960895F894FFCF67
:00000001FF
